:0400000011C0FECF5E
:10000400FDCF50C0FBCFFACFF9CFF8CFF7CFF6CF63
:1000140000000000000000000800040014000000BC
:10002400F894EE27ECBBE5BFF8E1A4B7A77FA4BF23
:10003400F1BDE1BD8DE0A2E0ED938A95E9F780E49E
:10004400A0E6ED938A95E9F7ECE1F0E0C8953196E6
:10005400802DC8953196902D0097B9F0C8953196AA
:10006400A02DC8953196B02DC8953196102CC89501
:1000740031966E2F7F2FF02DE12DC89531960D927C
:100084000197D9F7E62FF72FE1CFEFE9EDBFC4E7EA
:1000940040C0C498C3986880798048805980E1D072
:1000A400229608950A92AA93BA93EA93FA93EFB721
:1000B400EA93E0E0E2BFD8D0AE0EBF1EE62DF72DE6
:1000C400E370F070AE2FBF2FE1D060F4E0E9F1E00F
:1000D400EA15FB0538F4C498C398E4E0F0E06E2E0A
:1000E4007F2EBFD0E991EFBFF991E991B991A99120
:1000F40009901895CFD000E00E3140F4B8D01E2FEF
:10010400B6D0E11709F000E00F5FF6CFE12FC5D0BC
:100114000895E0E8E6BDE0E0E6BDE7E2E8BBE8E13B
:10012400E7BBE0E0EFBDE5E0E3BFE0E0E2BFE6BF50
:10013400E9BDEBBFE5BFE2E0E9BFE0E8E8B9E0E034
:10014400E3B9E9E3E1BDE9E2E1BD78942297E0E0B7
:10015400E883E983A895CEDFEF73E98362FE08C0E4
:10016400E981E770E33011F4662477242296EECF18
:1001740042FE07C0E981E07811F444245524229614
:10018400E5CF72D0E615F70519F4E981E27049F07C
:10019400E2E0F0E0E615F70519F4E981E17009F011
:1001A40003C06CD02296D2CFE62DE37009F43DC093
:1001B400E981E470C1F158D08E0E9F1EE62DF72D13
:1001C400E370E330F1F4E42DF52D309719F4E2E017
:1001D400E88316C0E130A0E0FA0739F4E4E0E883EC
:1001E400C498C39AE2E0F0E009C0E230A0E0FA0764
:1001F40039F4E4E0E883C49AC39836D04E2E5F2ED7
:1002040002C0E5E0E883E881A82DB92DF0E0AE173F
:10021400BF0710F033D007C0E981E47021F06ADF32
:10022400E983A895F9CF229691CFA895E981E37047
:10023400E03031F428D0C49AC39AE3E0F0E00CC073
:10024400E13029F420D0C39AE2E0F0E005C0E230C6
:1002540029F419D0C49A08D06E2E7F2E229676CF18
:10026400FFCF882499240895E1E0F0E008958AEC12
:1002740098E00197F1F7E6B3E7720895E4E0F0E05F
:10028400FA93EA9306CFAA24BB24EBCF00240A16E0
:100294000B0608951A930A930895099119910895E4
:00000001FF
